:1000000002780030B402D25202161F758C10D26BE7
:100010000214E730B502D25102169B32FFFFFFFFF8
:10002000FFFFFF32FFFF020032FFFF34344455561A
:1000300020208520F0E4787FF6D8FD85F02090E838
:1000400000E4F0A374EFB583F874F0B582F3A20373
:10005000920190006D75A0C078007402F208E493DC
:10006000F2A308046023E493F2A30880ED14D913EB
:10007000A024850629072D093321B10F831C661C96
:10008000461FD50A790A6AFFFFC20430961D3097D1
:100090001A7C14C296209713D29630970EC29720DE
:1000A0009609D297309604DCEAD204D296D2977D94
:1000B000177C2B0D90405375A0807800E493F2A339
:1000C00008B8000205A0DCF4DDF27583F41280604C
:1000D00090F408787775F003128079D200743F129B
:1000E000405290E7FE1240524017F0A3B403004084
:1000F00012124052400BF0A31240524004F0A38071
:1001000002C2001240527454124052122516122C90
:10011000887435122CA11219B950726F6772616D13
:1001200020636865636B73756D202D2D2D2D200068
:10013000E4FBFF900000C374532493FC7440341B11
:1001400004FDBC00011DE4932BFBE43FFFA3DCF6A0
:10015000DDF4A3A3E4932B7006A3E4932F600B12AA
:100160002C93121FC47590FD80FE121FB93000330E
:100170001219B94F7665726C617920726576697370
:10018000696F6E202D2D2D2D20200090E7FEE0249C
:1001900030A31219F4E02430A31219F4E01219F478
:1001A000121FCE7583F01280607583F41280609008
:1001B000F418788875F003128079745A1221B1749A
:1001C0001BFD1221B17493FC1221B19040530DE438
:1001D000931221B1A3DCF8DDF6E493A31221B1E47C
:1001E00093A31221B174A13002027461FE7C0079E4
:1001F000401221B11202251221CFF7543F09500AB3
:10020000F8EEC4440F68D36001C3EC92E303FC0E24
:10021000EE30E2DD90021DEC93F5778011030700CC
:100220000B0000000F7B127A00DAFEDBFC221219B1
:10023000B9546F74616C20706F72747320666F753F
:100240006E64202D2D2D202000AD770D7A00120A2E
:100250008E121FCE7436122CA112099CE577B404BD
:1002600000500302035824FD0303FCA20592F77912
:1002700040E70965F054806003757700DCF31219DC
:10028000B9536C61766520636F6D6D756E696361DE
:1002900074696F6E202D2000C3E5776006121FB9C8
:1002A000020358121FC47C0179401219B920536C03
:1002B00061766500AD047A00120A8EE76068F5F099
:1002C0001219B92020526F6D3A2000A2F012034497
:1002D0001219B9202052616D3A2000A2F112034494
:1002E0001219B92020492F4F3A2000A2F2120344DC
:0302F0001219B927
:1002F300202050676D3A2000A2F31203441219B96B
:100303002020547970653A200020F70B1219B94D5B
:10031300554C544900801D1219B950432F4D414388
:100323000080111219B920204E6F20726573706F0F
:100333006E736500121FCE090CBC04028017020203
:10034300AA40091219B94241442000221219B9479F
:100353004F4F440022E5777008122C9A7590FE8067
:10036300FE90E865F07437122CA112099C30030843
:10037300122FCF500302040675A0E97900906400A0
:100383007D017C507F007B00E493F3120416A309E4
:10039300B9000205A0DCF1DDEF75A0EA79009065F4
:1003A300007C00E493F579E493F3120416A309DCCB
:1003B300F61219B9436F6E66696720636865636BEC
:1003C30073756D20202D2D2D2D20009067FEE49355
:1003D3002B7027A3E4932F702190E900E0B4011A56
:1003E30090E901E0B4231390E902E0B4010C90E931
:1003F30003E0B40405121FB98030121FC47590FFC7
:10040300122CAE1207D54006122CB802037B122C15
:10041300BF80ED2BFBE43FFF220123010400051005
:100423000F2B78101A000021000090E904E0A2E0ED
:10043300923890E905E090E86EF0A3F090E906E0C9
:1004430090E86CF0A3F090E907E0F57790E908E015
:1004530090E863F090E909E090E86AF0A3F090E98E
:100463000AE090E868F0A3F090E90BE0F55F90E90B
:100473000CE0F57690E90DE0F57890E866F090E908
:100483000EE090ED00F030020990E865E0F57F02A0
:10049300253D1209A51280115389F0438901D28C9D
:1004A300D2A9D2AF755160755060755A40755940E5
:1004B300120629306E1F74201285521219B9504347
:1004C300206B6579626F617264206465746563741F
:1004D30065640D0A0012078312072D30251F1219B8
:1004E300A70D0A001219B950532F32206D6F75737F
:1004F300652064657465637465640D0A00206E038A
:10050300120691306E05121EE3C25C1280EAD268B5
:10051300D26E757B00757C0090E8577406F090E806
:10052300507400F0A3F0122CC9120A212001030217
:1005330005EA1219B90D0A5072657373200090050C
:100543008F122C2E9005A5122C2E2003581205581D
:1005530012056680561219A7656E746572206B6565
:100563007900221219D5656E746572206F6E206B47
:10057300657970616400223098FDC298E599221272
:100583002FCF400122B40702D322C322C04869748B
:1005930020656E74657220746F2070726F63656579
:1005A30064009320001205581205661219B92074CD
:1005B3006F20636F6E74696E75650D0A00E41240F7
:1005C3005243900320031212058240093098F81217
:1005D300057AB40DF2D2D1800E120582400930980B
:0105E300F81F
:1005E40012057AB40DF2437DC3C203E412405212E1
:1005F4004052A25D924AC25D1216FDA24A925D1259
:100604008520B3921B122C1A2000151219B90D0A59
:100614005374617274696E67206D61696E0D0A00AE
:10062400C201020AB6C2A8D21F90E88574FAF0E5A6
:100634005F540FB40548C2AA12079EC2B212022523
:10064400D2B3780F1285C17C05120225DCFBC2F0FF
:1006540090F401E030E02654E07900600279FF5321
:1006640082F8438203E0B900E720F00AB4FEE11205
:100674008ECFD2F080DA90ED00F012853422B404EB
:1006840008C2AA123FD7D2B32212077022206E7575
:1006940075B0FF7A0A7914E5B0543CF8E5B0543CDF
:1006A400687009D9F7E854246424600CDAE9121953
:1006B400B90D0A50430080537850D8FE7904B2B281
:1006C4007850D8FEA2B413A2B513D9F2D2B2B4CCE6
:1006D40014755F4412062912072D1219B94170705E
:1006E4006C65008026B488028003B4DD18755F55FC
:1006F40012062912072D1219A70D0A001219B9534F
:10070400756E0080061219B95043001219B9206B96
:100714006579626F617264206361626C65206465EF
:10072400746563746564200022C225C24DE55FB41C
:10073400550612079EC2AA22B44403C2AA22C24B7F
:1007440012079E12099C121A27121F232025143007
:100754004B19E55F54F0B4500122E55F540F442077
:10076400F55F22E55F540F4410F55F22752508D22A
:1007740088D2A8C289D2B2121EA64002D26E2275B5
:100784002608D2BAD28AC28BD2AAD2B312099C1238
:100794001EC34005D225121EC322E55FC45407754B
:1007A400F000B40304D2F08005B40502D2F07866F8
:1007B400C2F190F40012807990F41012807912073B
:1007C400C622D2EEF1CCC2EE79007A40D9FEDAFC30
:1007D400221219B952656C6F6164696E67204E56B6
:1007E40072616D20746F20666163746F7279206426
:1007F400656661756C740D0A00122CE11209337B75
:10080400007F0075A0EB790090041C7C00E4BC50D0
:1008140000502EBC40004008904052EC540F801B06
:10082400BC3000400474108018BC200040047401E3
:10083400800FBC100040047402800693BC0702E5DC
:1008440077F3120416A3090CBC00C29064001208CA
:10085400C350012290EB007C007412F0120416A322
:10086400DCF79065001208C350012290EB007C4035
:10087400E4F0A3DCFB7E08906600BE010E75A0EBDD
:10088400793EC3E49BF309C3E49FF375A0EB7900BD
:100894001214D95002D322DEE17B017E409068001D
:1008A400C082C083C0061208EBD006D083D0827504
:1008B400A0EB79001214D95002D322DEE3C3227CC8
:1008C4000075A0EB7900EC2582F582EC29F9C004CF
:0208D400C082E0
:1008D600C0831214D9D083D082D0044007EC2440C0
:1008E600FC70DCC322780490EB00D2217C00EC245F
:1008F6002B83F0BC081CBB00067D007A0180048BAC
:10090600057A00C000C006121FD5D006D0007C0BA9
:100916008002A30CBC10D70BD8D2C22122436F6D24
:100926007075746572202020202020202090094BAD
:1009360075A0EF7980E493F3A3097409B583F6747F
:100946009CB582F122C083C08290555574AAF0905E
:100956002AAA7455F090555574A0F0D082D083C061
:1009660083C082C0017C40E3F0DC02800409A380DE
:10097600F6C3F8E49368400430E7F8D320E7F4D0F0
:1009860001D082D0837C40E493F8E3A309B5000448
:10099600DCF5C322D32278007900D9FED8FC227474
:1009A600E61221B17C01EC1221B190ED00E0A31218
:1009B60021B1DCF990E9147E04120A1290E9247E32
:1009C60014120A1290EA047E24E578603790E93022
:1009D600E0FA8578F0A42404C39578F5827583EA55
:1009E6007C0C7905EE1221B10EE578B501005005B3
:1009F600E07A01800274121221B1E5822AF5820999
:100A0600DCE28003120A12E41221B1227C0CEE12FF
:100A160021B10EE0A31221B1DCF422E578B4020084
:100A2600402E7C01BC0400C00450098C747416125C
:100A3600813B80147401122130ECC412213074EF12
:100A46001221307416122130E578D0040CB504D486
:100A560022C0E0C082758205E4D5E0FDD582F9D0DA
:100A660082D0E02275F010A42400F582E5F0346807
:100A7600F58322120A6A5382C075A0EB79007C4086
:100A8600E493F3A309DCF922300124D22190E81083
:100A9600C004C001121FD5C2217C0390E810E012E9
:100AA6008552300003124052A3DCF3D001D0042259
:100AB600306B031214FAE55C7013304C05121EE31A
:100AC600C24C306D0812072D128E4AC26D122D0EC1
:100AD60090E866E0F578E55F540FB40416D55B310F
:100AE600755B10E5537003123E2CE55C7023123ED5
:100AF60088801EB40508121A01121A278013C24BE9
:100B0600121A27304B0BE55F54F0B420005002D286
:100B16006D205E0C20700C207109206F06020B6E92
:100B2600020D6CE55C6015207209D27290E83FE414
:100B3600F0803590E83FE0B40200402C7D03C2729D
:100B460030251574F5121E35206707121EC34002A4
:100B56008006DDEAC225C24DD27F75260885595A20
:100B6600755C00D25F1216FD30195C1221CF50570A
:100B7600F8128EAC120B7F804E30E73AB48008D262
:100B860068747E1285522230E617530007120F83CF
:100B96005407B40400502FE054F048F0F579D25DC4
:100BA6002230E505A2E0921B2230E41AD25C128EB6
:100BB6008FE8540FF0227583E8E575C4540F44405E
:020BC600F582B6
:100BC800E8F0D2752212864D4003020E08307A03EF
:100BD800020C6B30272090E850E0F8A3E0C868606A
:100BE8001375A0ECE2F556D27A08B8C0027800E88E
:100BF800F0020C6BC22720766AE550B5510280637B
:100C0800E55FB444028022B45502801DA851E6B4C1
:100C1800F706D211D2148007B4F80EC211D214E527
:100C28005104546FF551020D6C121A4930010F30FE
:100C38007A0CE556128EF27005E5571285341023AA
:100C4800028020E550B5510280F9121063128EB669
:100C580002203CE550B5510280F9121063128EBB98
:100C68000220F7307B11124052207B0830540512C5
:100C780013A0C254020D6C202747207C03020C905D
:100C8800122D1A403C020D6C203936307A33E55665
:100C9800B44A04D263802AB4CA1230631BE55F5495
:100CA8000FB40504D2538019D2768015B42D0930BB
:100CB8005306D276C2538009E4F57A522CC25EC23A
:100CC80053301907307A32C27A805BE5537050305E
:100CD8007A27C27AE55654FCB428258556F090E860
:100CE8002075552030F10574E0120D0330F00574BD
:100CF800F0120D03E557120D038069F0A305532286
:100D0800301810E556700CE557B4190040051281EB
:100D18003B8045128B01E553603E755520C27A75BC
:100D2800A0E8A855E2F830192A12217AE556128E61
:100D3800A77001F41221B1B4FF08E557A21892E692
:100D48008009E55654FCB4280FE557128EA21221EB
:100D5800B180051281C2400C307609E5537005C296
:100D680076020FCB307302802BE559B55A028024E6
:100D7800121C7E30011E30731B742012855274754C
:100D880012855290E82DE0128534A3E0128534A331
:100D9800E0128534E55C700F307365128CB6E55C43
:100DA800605E755E28C27375A0E8A95EE3F8301925
:100DB8004C12217A90F41A7415F07582187407F0A1
:100DC80090E828E0128EB11221B112217A5015B4A0
:100DD80080127C0390E829E0A3128EB11221B1DCC5
:100DE800F6755C0090F419E030E3FC30E2F990F419
:100DF8001A7415F07582187403F0020E0812821F17
:100E080012814C304F07302622C226C24F10592D6E
:100E1800105A3D10584F203D54105C15105D72104B
:100E28003C0C105B12105F12107509020F78020E4D
:100E3800AF020EEA020F38020EBD020EC7128E8FE5
:100E48005407303905A21BB392E7120EE0020F785F
:100E5800120F97203905B40302D23CA23992E71247
:100E68000EE0020F78E576120EE0020F7890E87730
:100E7800E004F0A2E01403C2E7900F8E93600840EC
:100E880002800874FC8004C23D74F4120EE0020F64
:100E980078203909E55F5407B40400500774F0124C
:100EA8000EE0D25A020F7874FAD1E0D23D90E8777A
:010EB800E455
:100EB900F0020F7874F1120EE0D258020F78302543
:100EC9001385595A121F9B74F4121E352067051297
:100ED9001EC3C27F020F78C226121DE6D24FD26A04
:100EE90022128E8FF8E55F540FB40407E8124024EC
:100EF900020F78B40525C000780E1285C1D000E82C
:100F0900A2E092F2A2E192F0A2E292F3A2E392F1BC
:100F190053F00FA8F01285C1020F787D0A74ED1203
:100F29000EE0303905306602DDF3D259020F7875CB
:100F390083E8E575C4540F4440F582E0F8E55F5451
:100F49000FF9E579540FB404028024B40512B80EE0
:100F590003020EEA203912B90515E81285C1800F7E
:100F6900B8ED03020EEAB9ED06E8120EE08000C200
:100F790075205E03020AB6020FDB7583EAE5764443
:100F890000F582E022391911125914765800E579D1
:100F990054077802B4030040027803E55F54FC4526
:100FA90000F55F30391AE579D2F054F06002C2F0E9
:100FB900E57954077803B404005005A2F092E422BD
:100FC900E82290E873E551F0757E00D25E90E884DE
:100FD900E4F090E884E0B42003021106C3E550244C
:100FE900109551540FF8E55F540FB4041BB8020073
:100FF9004059121063FE12106330E74CCE20E748C7
:1010090053067F6E7042803BB405234021B803002C
:101019004039121063FE12106330E72CCE20E72806
:1010290053067F6E7022121063B47F1C8015B803BB
:10103900004018121063FE121063B4F00B12106313
:101049006E7005121070704C02110FE86009A851FA
:10105900860612107060F1020AB6A851E6128ECA0D
:101069000853006F885122EE121A4C307A1DC27A49
:101079009011637C008002A30CE4936016B556F7C7
:10108900901182EC93B43105200008E42250042029
:1010990000F91422BC0A005036E57E75F00AA42C2A
:1010A900500205F0F57E85F07FE52C5407701D058B
:1010B9007AE57AB4020AE577B46300500F02112287
:1010C90050FBE577B409005003021122020FD6BC88
:1010D9001100500874F72C422C020FD69011A0EC85
:1010E90024F6230493C0E0EC24F62393C0E022C342
:1010F90078007908102605D8FBD9F9D322E52C54B4
:1011090007700302112290E873E0F551755800E465
:10111900F57A522CC25E020D6C1211404016F57E12
:10112900E577B57E00400D857E76C238C270D26FF4
:10113900C25DC25C020CC0857FF0E5F0B4020050CC
:101149000CE57E20F005600514C32260FBD3224420
:1011590010F0A3F0A3EEF0A3F0223031323334358E
:10116900363738397674706D61777573786B473BAC
:101179003A43726E69642E0C0032323232323232A4
:101189003232323230303030303032323232323242
:101199003232323231313211C811CD11DA123311F2
:0111A900E95C
:1011AA001206121A12DC12E1139A12FC12E612F05B
:1011BA0012F4130B135E134B1345133B132890E8D9
:1011CA0068800390E86CE57FAE7E121158020CC06D
:1011DA001211404051604FF5771216FD020CC0E51E
:1011EA007F7043E57EB48000503CC082C08390E8A3
:1011FA0063F0D083D082121F10020CC0E57F7026E4
:10120A00E57EB40200401F90E930F0D26F020CC0B4
:10121A00E57F7012E57EB41100500BF57890E86610
:10122A00F0D26F020CC002110FE57F701FAA7EE593
:10123A007E6019B40B00403CB41400400FB4160091
:10124A00400DB41E004005B421004012020CC0E556
:10125A007EA2E0E55FC2E392E3F55F020CC0E55FC0
:10126A00540FF9E57E24EB834501F55FD26D020C3C
:10127A00C0102050120F83BA04047444803EBA0589
:10128A000474558037BA0B0474668030BA0C04743F
:10129A00778029BA04004013540FCA24FBB404040B
:1012AA0074058016B405137400800FC4540FA8790E
:1012BA00530007B8040040027401C44AF579D25DAC
:1012CA00120F83E579F0FBD24AE582FE12249D02D1
:1012DA000CC0D238020CC0C238020CC0D270C2385C
:1012EA00C25DC25C8009D27180F4A201B39201028C
:1012FA000CC0E52C540760062409FC0210E5021113
:10130A0022200003122510121959C238E55FB4448D
:10131A000280DCB4550280D7D24CD26D80D1300025
:10132A000AD27CD27B124052020CC0122E15020C39
:10133A00C0D27BC27C124052020CC0124052020C34
:10134A00C07E00902537EE936007FA121C460E8085
:10135A00F2020CC0121364020CC0E579540FB404F3
:10136A0000501120180F201921E574D2E212847B53
:10137A00E41284B522E57412847B74EF1284A4E526
:10138A007412847B74311284A422743112213022A3
:10139A001213A00212F91213A912141A500022E50C
:1013AA0078606C7B00EB12847BC023C21974EF1245
:1013BA0084A4EB12847B74151284B5D0230BBB046E
:1013CA00028006E578B503DD22E57824FC6040FB5F
:1013DA00757540D219D2187401122130E57512219F
:1013EA0030D2237415122130E5752410F575120ACE
:1013FA0057DBE47416122130121782120A57120AA6
:10140A0057120A57120A57120A57120A57D26F224C
:10141A0090E86EE090E905F090E86CE090E906F05B
:10142A00E57790E907F090E863E090E908F090E842
:10143A006AE090E909F090E868E090E90AF0E55F6F
:10144A00B444028003B4550474128002C2E090E9E5
:10145A000BF0E57890E90DF090ED00E090E90EF0E0
:10146A001209337B007F007C5090E900E493120458
:10147A0016A3DCF875A0EB790090EA007C00E493EF
:10148A00F3120416A309DCF690640075A0E979004A
:03149A001214D950
:10149D0050012290644075A0E979401214D9500191
:1014AD00229065001208C350012290EB007C40E4AD
:1014BD00F0A3DCFB90EB3EC3E49BF0A3C3E49FF0F1
:1014CD009067C075A0EB79001214D922128A1D12F3
:1014DD00EF8092F01289F2A2F022202B06107E03EB
:1014ED00752508203306107D0375260832C26B3032
:1014FD003B12C3E55024109551540FB4090050040C
:10150D00D2B2C23B303A16C3E5592410955A540F46
:10151D00B409005008D2B3C23AD249802F90E87670
:10152D00104927E004B408004021755C00E55AB568
:10153D0059028016F8E6B4AA0E0853004FE670075C
:10154D0085595AD26D800385595AE4F012405210D4
:10155D006A11304F0EC24FC259C25AC258C25CC234
:10156D005DC25B203932307917307710121846740E
:10157D0031124052124052C277122C1AC279801287
:10158D0090E8691215F6501012181CD277124052BD
:10159D00800690E8681215EE90E884E004F090E87B
:1015AD003FE004F012855D20111F201A1C207B19CD
:1015BD0030381690E86D1215F6500ED215D270C255
:1015CD005DC25C90E86C1215EE303F1190E867E05B
:1015DD0004F0B402004006121879122EEA122EF70A
:1015ED0022E0A3F0A3E0A3F022E02410F0501FF8B6
:1015FD004410F0A3A3E0B80002601314F0B4FF0987
:10160D00E81415821582F0C3227003E86002C3222C
:10161D00D322202F1E302B0A105272D279D27E1572
:10162D002532C55203D2E7105202C2E7C552152525
:10163D00C22B32102844752508105203D274323053
:10164D0013FAC2B2C001C55264FA7008D226C5524F
:10165D007930801F64FAC552A950A7520953016F02
:10166D008950C904546F65517006D23BC9D00132FF
:10167D00C97926D9FED2B2D00132C552D213105239
:10168D000520D007800330D002C213C55232203757
:10169D002030330C105108D279D27DD24915263223
:1016AD00C55B03D2E7105102C2E7C55B1526C233F5
:1016BD003210302875260810510132306C31C001BE
:1016CD00A959A75B0953014F8959C24BC904544FFE
:1016DD00655A7004C2B3D23AC9D00132C55BD26C1F
:1016ED0010510520D007800330D002C26CC55B328B
:1016FD00205E27205924205A2120581E203D1B20D2
:10170D005C18205D15203C12205B0F10700D1071C0
:10171D0018C26FE577B57600501B220576E577B5D3
:10172D0076005011757600800C1576E576047005FF
:10173D008577768000C20774AA42C0D21F1289B97C
:10174D00123062203903124052204E0312187912C2
:10175D001782304E0D1219A72066702A00C218C2CA
:10176D0019221218F71218B2123069101501223011
:10177D001402D25B22A976121799F575A2F6921969
:02178D00A2F7C1
:10178F009218A2F5924E12869922203904E57870AC
:10179F0006E9C454F0802EE578B40F03E98026855E
:1017AF0078F090E930E0A414B50100500BC304F5B4
:1017BF00F0E995F0257880DA90E930E0F5F0E984EA
:1017CF00540FC445F0F875F00020390BE854F0C4FD
:1017DF00B578005002D2F7E854C06002D2F6C0F0DC
:1017EF0090E930E08578F0A4C0E0E5F06006D0E045
:1017FF00D0F0E82290E865E0D0F025F0C39578B5F9
:10180F0001005005D0F0D2F522D0F0E822201805C3
:10181F0020191C801FE575C4540312847B74EF12CA
:10182F0084A4E575C4540312847B74021284A474D7
:10183F0002122130C2EC2220190520180280283014
:10184F001905740C12213030181FE575C45403129A
:10185F00847B74EF1284A4E575C4540312847B74E3
:10186F000C1284A4201902D2EC22C23F20191F307F
:10187F00182EE575C4540312847B74EF1284A4E50B
:10188F0075C4540312847B74161284A4801230180A
:10189F000A74EF122130741612213074161221308F
:1018AF00C2EC2220183C30192F740912213012215A
:1018BF008FD268F854706020C4B40600501AE8A2A2
:1018CF00E7921B128E8FE8540FF0E8C45407F812FA
:1018DF000F8354F048F08003120F83F579D25DD255
:1018EF005C22120F83F5792220182320190EE5753B
:1018FF00C45403F57444FCF590D2EC227401122108
:10190F0030E57554F0122130740C12213022201959
:10191F00241218FDE57412847B74EF1284A4E5740D
:10192F0012847B74011284A4E57412847BE57554D0
:10193F000F1284A42212190B74EF122130740112AA
:10194F002130E575540F1221302220181020193A3A
:10195F00909285E574540393457DF57D22301903EC
:10196F00121999E574540312847B74EF1284A4E561
:10197F0074540312847B74301284A4E574540312DC
:10198F00847BE575540F1284A4227430122130E544
:10199F0075C4540F12213022D083D082E493128564
:1019AF0052A3E493B400F7740173D083D082C08242
:1019BF00C083E493128552A3E49370F8200007D0FC
:1019CF00E0D0E0740173D083D082E493B40A028034
:1019DF000D30010A300007C001124052D001A3E4BC
:1019EF009370E904733001091285523000031240DD
:1019FF00522290F401E030E01E54E0790060027949
:101A0F00FF5382F8438203E0B900E7A950F705506E
:101A1F0053506FD27980DB2290F411E030E01A53EB
:101A2F0082F8438203E0A959F7128F0B05595359D6
:101A3F004FD24BD249D27980DF22121063F8FCAE1D
:101A4F005F53060FBE0402804DBE05028048E55865
:101A5F006003021B37B8AA06D26E121EE322B8DF4C
:101A6F00004033B8EF16D2397430124052757800F7
:021A7F00D22370
:101A8100C23875770FD26ED22522B8F0047558018D
:101A910022B8E00475580222B8E104755804227591
:101AA100F0008062E55F540FB404059022F2804893
:101AB100B405059023728040C392F0E55F54039012
:101AC10021DF7885B40305902264788EECB500009F
:101AD100503493A87920391CB844028003B85514B6
:101AE100A85F53000FB80A00500AB44C02741BB42B
:101AF1004B02741EA2F08006E8A2E7C2E79364FFDE
:101B0100701C92F0C2F1E55F647954036027742878
:101B1100A2F092E0A2F192E1F5568C57801264FF97
:101B210030E70975560092E7F557800492E7F556BC
:101B3100D27A75580022E558B401028012B4020429
:101B4100C2F0800FB40305D2F0021B5C021C1CD34F
:101B5100021ABAE8B4F00475580322901B97E4A363
:101B610093A36015B500F7E49330F0022402F55712
:101B7100755600D27A75580022901B9DD2F1787F5C
:101B8100ECB50000508093F5567003021B0730F04E
:101B910003435680021B311201590200000000006C
:101BA100000000000000000000000000004D0000E7
:101BB1004B000000000000000000004E000000008B
:101BC1000000004F000000000000001D00000000A8
:101BD1000000000000000000000000000000000004
:101BE1000000000000005B00000000000000000099
:101BF1000000000000005F00000000000000000085
:101C010000000000005300585200000050515700DE
:101C110059560000000055000D547E901C3AE558BD
:101C210093B500150558E5589370117A0F121C46AB
:101C3100742D121C668002D27A755800221477E145
:101C4100F014F0770090E850E0F875A0ECEA7C021F
:101C5100B42D027C01F208B8C0027800D2E7DCF5AD
:101C6100E8F0D22722C0E090E850E0F875A0ECD06F
:101C7100E0F208B8C0027800E8F0D22722E5592442
:101C810010955A540FF8E55FC4540FB4040AB80212
:101C910000403F121CD48038400CB805004033127C
:101CA1001D0F402E802A204B1F303908E57954F052
:101CB1006005800A304D07B8040040168005B8035E
:101CC10000400F128D938008B803004005121D7863
:101CD100D27322A85AE60853004F885A75F008A219
:101CE100E7B392F0A2E692E7F404A2E792F590E856
:101CF1002FF0A85AE60853004F885AA2E692E7A2AD
:101D0100E792F490E82EF090E82DE5F0F02275F0DE
:101D110008A85AE630E74EF4A2E292F0A2E192F26C
:101D2100A2E092F10853004FE6FE080853004F2647
:101D310090E82EF0EE6630E701B392F41853000FED
:101D4100430040E6FE080853004F2690E82FF0EECE
:101D51006630E701B392F50853004F885A90E82D99
:101D6100E5F0F0C3220853004FC3E559986004E63B
:031D710030E7F266
:101D7400885AD32275F000A85AE630E65308530077
:101D84004FA2E592F0A2E492F1A2E192F4A2E392CE
:101D9400F5A2E092F2A2E292F3E60853004FA2F217
:101DA40092E6C392F2A2F492E790E82EF0E608538A
:101DB400004F885AA2F392E643F008A2F592E7F4A2
:101DC40004A2E792F590E82FF090E82DE5F0F022D8
:101DD4000853004FC3E559986004E630E6F2885A88
:101DE400D322128ECF128A1D303B03D3803D7F3C19
:101DF400DFFEC266C2B4D2B2A2D0B37C097E0A7F2F
:101E04000030B210DFFBDEF9D2B4D26680DD121EE0
:101E14007A2066171392B4121E84DCF2121E7AD250
:101E2400B4121E84121E7A121E84C3D2B41289F212
:101E340022128EE3128A1D303A0AC23A855A598018
:101E4400F3D3802C7F3CDFFEC267C2B5D2B3A2D0ED
:101E5400B37C09121E8E2067171392B5121E9CDCE8
:101E6400F2121E8ED2B5121E9C121E8E121E9CC31E
:101E7400D2B51289F2227FFF30B204DFFBD2662290
:101E84007FFF20B204DFFBD266227FFF780830B3E5
:101E940006DFFBD8F9D267227FFF20B304DFFBD231
:101EA400672278007908E550B55106D8F9D9F7D3F7
:101EB40022A851E6128ECA0853006F8851C322E447
:101EC400F8FE7902E559B55A08D8F9DEF7D9F5D301
:101ED40022A85AE6128EDE0853004F885AC322E520
:101EE4005F5407B4040040012274FF121DE63066FB
:101EF40001221210F840FA7A017C00121EA6500446
:101F0400DCF9DAF7121F10D25CD25D2274F3121DD1
:101F1400E61210F890E863E0121DE61210F822C2EF
:101F240025C24D85595A74FF121E3530670122129D
:101F34001EC340627C03121EC364AA6002DCF71253
:101F44001EC3901F60E493601774F3121E35121EB3
:101F5400C3E493A3121E35121EC380E9C864500063
:101F640074F2121E35121EC3121EC3C24D6002D279
:101F74004D74E8121E35121EC37403121E35121E50
:101F8400C374E6121E35121EC3121F9B74F4121E74
:101F940035121EC3D2252274F3121E352067151282
:101FA4001EC37428A8795300F0B850027414121E8A
:101FB40035121EC3221219B9474F4F440D0A00228D
:101FC4001219B94241440D0A00221219B90D0A002E
:101FD4002275A0E87959E4F319F37C10C3ED33FDBD
:101FE400EA33FA75F002A801430001E235E0D4F2C5
:101FF40018D5F0F7DCE675F003A801D375A0E8E284
:1020040030F003088001C4540F500D700A20F2030D
:1020140030F10574208003C34430302104F0A380E0
:102024000E305608101E08122C338003128552D528
:10203400F0CA302102E4F022301736C217547FF878
:1020440090E85CE0540FF94400F5827583EAE8F007
:10205400E9B576048879D25DB90400400D7440492D
:0320640012213016
:10206700E0122130020D6CE81280B7020D6C30E6E9
:102077000990E85CF0D217020D6CB4160AD23F90B3
:10208700E867E4F0020D6CB4010B303F03121879D6
:10209700D21D020C5BB40C08121846C21D020D6C4F
:1020A700B4020812181CC21D020D6CB415030213EA
:1020B7009AB43106121364020D6CB43007D248C2C9
:1020C7001D020C5BB408087490121DE6020D6CA289
:1020D700E792F0C2E7B419004013B42F00500EA2E4
:1020E700F092E7F557755600D27A020D6C020D6C27
:1020F700301D10540FF576C271C270C21D1216FD45
:10210700020D6C304811C248D26DB40400500B90D8
:10211700928593457DF57D020D6CC0E074301221E8
:1021270030D0E0122130020D6C200209F82023067E
:10213700B4EF03D22322302403FF8016B4010280B8
:102147000CB430028007F85300F0B84004D224FEE4
:1021570022FE12217AE41221B1EEA22392E7128E17
:10216700C01221B1302407EF128EC51221B1C2234C
:10217700C2242212218F5009B48002D322B48102D3
:10218700D322F8120B7F80EBC310681DC000C0017B
:10219700780079141221CF4006D8F9D9F77404D002
:1021A70001D00030010312855222C0E075A0F478F7
:1021B70019E230E2FCD0E0781BF22275A0F478191E
:1021C700E230E0FC781BE22290F419E020E003C340
:1021D700E42290F41BE0D322FF09FF050301020C60
:1021E700FF0A080604462FFFFF4C48FF4A7131FFDC
:1021F700FFFF7A73617732FFFF637864653433FFDB
:10220700FF447666747235FFFF6E6268677936FF42
:10221700FFFF6D6A753738FFFF416B696F3039FF14
:10222700FF42436C3F703AFFFFFF40FF3C3BFFFF1D
:102237007C49473DFF3EFFFFFF1CFFFFFFFF45FFB8
:10224700FF11FF1417FFFFFF1060121516182E7BE2
:102257000B5E135D5C190EFFFFFFFF077DFFFFFF9E
:10226700FFFFFFFF012EFFFFFFFF462F02FF4A4838
:102277001C7C713103FF4C7A7361773204FF6378FA
:102287006465343305FF44766674723506FF6E6203
:102297006867793607FF4D6D6A75373808FF416BF8
:1022A700696F303909FF42436C3F703A0AFFFF40BC
:1022B700203C3B0B0D4B49473D3EFF0C0E57580F3B
:1022C7005651534550FF1159141755525410601267
:1022D7001516187B5BFF5F13FF5E195CFF1B1EFF64
:1022E700FF5DFFFFFFFFFFFF4E4F1D6173646668D1
:1022F700677A7863761C62717765727974313233E5
:102307003436353B39373A38303D6F753C6970475D
:102317006C6A406B3F3E41436E6D4246442F45FF1A
:102327002E4A4F481A4C58595756FFFF60FF5CFF1B
:102337005EFF7BFFFFFF5B5FFF5DFFFF99101112E1
:102347001314151617FF1819FFFFFF0506070308D3
:0B23570009FF0BFF0DFF0EFF0AFF0C3B
:10236200FF0F505254510453025501494D4BFF1F68
:10237200FF9E9C9F9D01020A030B040C054D06A9BA
:102382000708094C560F0D0E58A0A157592E31328D
:1023920033343536373839303A3B2F45509B5B5C06
:1023A2001FA260A3524671776572747975696F7066
:1023B2003C3D514B1718195DA4A553FF4A61736444
:1023C2006667686A6B6C3F403E475F14151610A63D
:1023D20054A77B487A786376626E6D41424349FF27
:1023E200111213AAABAC9A7C4E444F551C5EFF2DC2
:1023F20044B1C0B3B4B5B740B9B0B8BB413A424337
:1024020030313233343536373839BF3FC13BC2C33E
:10241200B2E1E2E3E4E5E6E7E8E9EAEBECEDEEEF70
:10242200F0F1F2F3F4F5F6F7F8F9FA3C3E3DB6BAFC
:102432002F6162636465666768696A6B6C6D6E6F53
:10244200707172737475767778797ABCBEBDAF1B82
:1024520060303132333435363738392D3D5B5D5C8F
:102462003B272C2E2F2008090D1B7E2921402324D7
:10247200255E262A285F2B7B7D7C3A223C3E3F202C
:1024820008090DB576048B79D25D7583EA4400F5AF
:1024920082E0B503028004D254EBF0EEF9121799F0
:1024A200F920F71F20F60DE9C45403F9EB1280B7A7
:1024B200D26D8041E9C4540F4440122130EB122105
:1024C200308032E9C45403F8E9540F4440F943031D
:1024D2008030F60F74EF122130E9122130EB122115
:1024E20030801274EF1224FEE91224FE74EF1224DB
:1024F200FEEB1224FE204A03123D1522C0E0E81230
:10250200847BD0E0C023C2191284A4D023221219E2
:10251200B90D0A001219B950726F6772616D20729B
:1025220065766973696F6E202D2D2D2D20553434FB
:10253200440D0A0022733434642D0090F0007C07AD
:10254200786675F0011280795382F8E5822408F5E5
:1025520082BC040390F400DCEC90F4187888D2F189
:1025620012807953A8FA1219B9446961676E6F73C0
:10257200746963206D6F64650D0A00903BBC122C78
:102582002EE57F0404FC7483122C44902A31122C11
:102592004BD20D5389F0438901D28C903BA6122C69
:1025A2002E902A4B122C2E200D0A74201221B1904B
:1025B2002A47800874101221B1902A43122C2EE56A
:1025C2007F04B40203E480050303145403F5487541
:1025D2004900754A007549007590FCD2EC200D0542
:1025E2001226D08003122638C2EC122846E549652D
:1025F2004805496014743045491221B17C0679407E
:102602001221C2F709DCF980E1054AE54AB4640304
:10261200754A0074C0122C447A00AD4AD21ED256BA
:10262200121FD5C2560547E547B46408D20C90F88C
:10263200007408F0809FD202B2027B0375464020EC
:1026420002081229A012283880031229AE7C047ACB
:01265200FB8C
:1026530080097546407C087AFE0546200203630222
:10266300FFEABB0406F5C0E5C0800E500844C3F57D
:10267300B0E5B08004F5C8E5C86A8A003002036398
:1026830000FF55006004A84646F6E5D8540F6002E3
:102693004243E590543C643C600242447E0475A08E
:1026A300F07819122829E824F8F8DEF775A0F478F1
:1026B30011122829EA23FA122952DCA50B1229C781
:1026C300122818BB068F3002012202263AC20212D8
:1026D30029AE1228187C047AFB7B03E41228388085
:1026E300067C087AFE79FCEABB0408F5C0E5C0A8BD
:1026F300C8801B5013F5B0E5B044C37F001228DF38
:10270300BF0101F442408022F5C8A8C8E5C07F009C
:10271300491228DFC8491228DFC8BF0106F449C897
:10272300F449C8694241E8694242EA23FAEC30E0DD
:1027330007E92323F9122952DCAD0BBB06A375C0AD
:102743000075C800E5D8F4540F6002F5437C04908B
:10275300F01B785AE8F023F8E58224F8F582DCF4DC
:10276300C2EE90F403E8F01229BD1228187C047815
:102773005A90F019E030E00F05820582E0158215CA
:1027830082B50003C38001D3E54533F545E58224D3
:10279300F8F582E823F8DCDCE545C333F54590F42E
:1027A30011E030E00905820582E0650060034345DE
:1027B30001D2EEE590543C643CF544A202920ED261
:1027C30002D2EE1229C7E590F4543C643C42441211
:1027D300281890F411E020E70BC2EE1229BDE03077
:1027E300E7028003434402C2021229AE122818C230
:1027F300B21229BDA20E9202783A122A6890F4010D
:10280300E030E00A05820582E0B43A0280034343E4
:102813001012281822E5905403B40307C2EC7590F4
:10282300FC8002059022E254F1B40100B3E5457245
:10283300E433F54522E4F540F541F542F544F5432B
:10284300F54522E5415542FD9028727C045403B4BA
:102853000313E493A3FE7F5812292DD20FE493525E
:102863004152428001A3A3ED0303FDDCE080080293
:10287300FC01F303CF043F902A097C14E5400303D2
:10288300540FB40F0D7E007F58D20F902A117C1184
:102893008013BC1004E5418005BC0802E54213FD2A
:1028A300500D1228EB12292D122942D20F8002A3B8
:1028B300A3EDDCDE300F05122942C20FE5436006AB
:1028C3001228F4122942E544600703122918122939
:1028D30042E545600612291C1229422275F008338D
:1028E30040010FD5F0F93322E493A3FEE493A3FF51
:1028F30022FD30E4077E007F5312292DED7F42F540
:10290300F0A2F092E1A2F192E0A2F292E3A2F3929A
:10291300E27E0180087F4480027F507E00135005D1
:10292300FD12292DED0EBE05F422E5496006BE0019
:102933000122232324C32E122C44EF122C3322D240
:012943000F84
:1029440079C0E4D9FEC9122952C9D5E0F622122968
:10295400844004C2068016200613D206100C0F759C
:102964004700B40702B20D75810702259522C08382
:10297400C08290F800740CF0D082D0837547002296
:10298400C006C002C001C000C083C082122FCFD0D5
:1029940082D083D000D001D002D0062275B0C3E427
:1029A400F5C0F5C8D2EE1229C72275B0FF74FFF541
:1029B400C0F5C8C2EE1229C72274127900D9FED517
:1029C400E0FB227C0875A0F07802BC040775A0F433
:1029D4007802800ABC03028025BC010280207402B4
:1029E400F2200204747080027460F27445F21229B9
:1029F400BD18E230E0070808E2181880F508E8245A
:102A040008F8DCC6220037003900380041024102D0
:102A140039014101390341033904410439023802BF
:102A24003701380137033803370438043743313268
:102A34003334353637383930313233343536008033
:102A44004F5000804C4200C02030004C4F4F50008B
:102A54004F50454E000D0A0020504153530020466C
:102A640041494C00C3122A7A7C08E813122A7ADC02
:102A7400FAD3122A7A22CA858AF020F7FA858AF0D4
:102A840030F7FAB392B2858AF020F7FA858AF030EB
:102A9400F7FA858AF020F7FA858AF030F7FACA2225
:102AA400E4936006A312855280F622E549600B90F8
:102AB4002B757C04232304FD8019902A54200D03D4
:102AC400902A4F122AA4902A59122AA4902B597C96
:102AD400057D00E57FB401021C1CC083C082C001D7
:102AE400C004C0057A00D22190E810121FD5C2217B
:102AF40090E811122AA4D005D004D001D082D0834A
:102B04000D7907C3E493A3F8E493A3566024400F1C
:102B1400C083C082902A62122AA4D082D083D37444
:102B240020128552E493A3128552E493A312855292
:102B34008002A3A3D9CE400CC083C082902A5C1229
:102B44002AA48004C083C082902A59122AA4D08265
:102B5400D083DC86224004303740103038400830BF
:102B6400394020313044023133450132354310516C
:102B74003142083037420430384108303941043199
:102B8400304302313144043133450232354201309D
:102B9400374202303841013039410231304301318A
:102BA4003144083133450432354220303742103045
:102BB400384120303941103130430831314410312B
:102BC4003345083235428030374240303841803016
:102BD40039414031304304313144203133451032DE
:102BE4003590F8007430F07406F0740CF02290F80C
:102BF40000740DF02290F800740CF02275A0F8799E
:102C040000F30975A0F87901E493A36008B45C02A9
:102C1400748CF380F322207710903BFE201B0390EA
:102C24003C14122C2EA21B921C22E493A380CD757B
:022C3400A0F806
:102C36007901645C6004645C8002748CF32275A084
:102C4600F87900F32275A0F87901E493B45C027474
:102C56008CF3A3DCF5227480122C44E576122C7FCB
:102C66007420122C337A00AD760DBD00047A017DF6
:102C760000D256121FD5C25622120A6A7C10122C96
:102C86004B2290F40F7403F090F41FF022903BD285
:102C9600122C2E22903BE8122C2E22C0E0749312A6
:102CA6002C44D0E0122C3322903B90122C2E122C66
:102CB600F322903B38122C2E22903B64122C2E12BB
:102CC6002CF3229030701231C2D21690E85F7479DC
:102CD600F090E85E122F7112311E22903B7A122C70
:102CE6002E903BA6122C2E74C0122C4422903B4EE2
:102CF600122C2E122D05122FCF50FBB407F82212DC
:102D06002FCF40FB123D0C22305708C25720390303
:102D16001232A022E5536002D322307A10AE56BE9C
:102D26002E0EC210C27CC2507C2D122E69022E06B7
:102D3600201042BE79217C22122E69C250D21090F8
:102D4600E8377401F090E838E0123CD97C10742022
:102D5600F0A3DCFC022E06BE6ED390E838E004B584
:102D6600770280034001E4F07C2D122E69122E2A90
:102D7600C27A022E0A7445A879B855027451B5066E
:102D86001390E837E0B40102807614F0123CD9744F
:102D960020F0D322BE4718123CF6C21090E838E065
:102DA600B57603122C5C90E837E0240AFC80BBBEA3
:102DB6004804D250D322BEC804C250D322BE8000DB
:102DC600503CBE2E004039BE4800500E903D9B3010
:102DD6005003903DB5EE93FE8011BE7B005021BEA0
:102DE6006100401CEE30500324E0FE90E837E064BA
:102DF60011600D123CD9EEF090E837E004F0D322D2
:102E0600C27AC322E4F52CF57AC25EC253D322D22B
:102E16007C90E838E576F0C2507A48121C46122EAD
:102E26002A022E0A90E838E0FF903C8C122E93D2AC
:102E360021EF2401FDE43400FA90E83B121FD5E4AB
:102E4600F090E83B122E93C221903C91122E93EF04
:102E5600120A6A7C10122EA3EF120A79903C951280
:102E66002E932290E850E0F875A0EC7445AB79BB40
:102E760055027451F2D2E708B8C0027800F2C2E7F0
:102E860008B8C0027800DCECE8F0D2272220210442
:102E9600E4938001E06005122EB180F12220210426
:102EA600E4938001E0122EB1DCF322C083C082904D
:102EB6003D4A93FA53027F20E70C305013C25074F8
:102EC600C8121C66800A205007D2507448121C662D
:102ED600C004121C46D004D082D083A322903CC3E7
:102EE600122C2E22903CAD122C2E903BBC122C2E76
:102EF60022201169201A41203E02801090E853E0FA
:102F0600B41E0040051230B4800204F0201A2920B5
:102F1600191330180A123D48A2E7B3921B80061215
:022F26003D5616
:102F2800B3921B201C05301B0D8003201B08303971
:102F380002D25C122C1A122F8A9257501E90E85314
:102F4800E4F0D27990E85F7479F090E85E30221965
:102F580090F800740CF0C257C2222290E85DE01489
:102F6800F0701EA3E014F070187404F015827484D5
:102F7800F090E85FE014F0700890F8007408F0D260
:102F88002222122FCF4008C20690E856E4F0229081
:102F980030229360F214FE3006028004D3D2062257
:102FA800BE0B02800DBE0C028008BE0E028003BE5E
:102FB8000F1390E856E00430E30A2408B4280050C0
:102FC800DBF080D8F0C32275A0F47583F4780D790E
:102FD8001D75820E7A0112300FB40F2975820E7A90
:102FE8000212300F2410B41F1C75821E7A01123091
:102FF8000F2420B42F0F75821E7A0212300F24304E
:10300800B43F02C322D322EAF0E25403FEE354039E
:10301800232342060582EAF0EE22000000000000A9
:10302800000E00000008000502000000000000007B
:103038000001000000090006030000000000000075
:10304800000F0000000A0007040000000000000054
:1030580000100000000D000C0B00201A03122C5C5D
:1030680022201A03122C1A22BE0B0BD270D215C2C0
:103078006FC238023117BE0C0BD271D215C26FC2A3
:1030880038023117BE0A2290E835E4F012327C90FB
:103098003C2A122C2E122BF9D21AC26FC271C2709E
:1030A8009031D11231C2023117BE0D15C23EA81F90
:1030B80012312D403B122BF97491122C44122C6BB7
:1030C80022BE0A004006203E0302316FD23EC238BB
:1030D800123614122BF2E51FB43D09E577B46300EC
:1030E800500D800C500AE577B40900500280012287
:1030F800C23E1231544007B57702800740051230AE
:10310800BD800CF576C270C271C238D26FD215126A
:10311800311E122BF922E490E853F0A3F0A3F075C6
:103128001F3BC23E22B83B02C3227E0090E83BE030
:10313800CE75F00AA42E500205F0FEA318B83BEF96
:1031480090E854F0FDA3E5F0FAF0D32290E855E0BA
:10315800F5F0B40200500E90E854E020F005600548
:1031680014C32260FBD322C23890E854E576F0906D
:10317800317D1231C290E854E0BE0D0DD26FD215E8
:10318800F5769030701231C222BE0E0814B4FF10CA
:10319800E577800CBE0F1904B5770280034001E47F
:1031A800F0AF76F57674C0122C44122C618F76221B
:1031B800122C1A9030701231C222C083C08290E85B
:1031C8005AD0E0F0A3D0E0F02290E835E0F8BE0B4A
:1031D8000704B40E0CE48009BE0C2614B4FF027474
:1031E8000DA95F530107B40D05B905E28010B404B9
:1031F800028008B40C028003B40B03B902D0F0803B
:1032080073BE0A58105415C21A9030701231C21287
:02321800311E65
:10321A00122C5C122C1A122BF922903C40122C2EE2
:10322A00903C56122C2E90323C1231C290E835E472
:10323A00F022BE0B028003BE0C1290E835E0F4F0D7
:10324A00903C6C6003903C71122C2E22BE0DFC90B7
:10325A00E835E070B01213A080ABBE0DBCE823F8CD
:10326A0090387E93F9A3E893F58289831231C202DA
:10327A0032A090E835E0F875F014A4244DF582E503
:10328A00F03439F5837480122C447C14122C4B12BE
:10329A0032AB1232B42290E85AE0C0E0A3E0C0E0B8
:1032AA0022903902E893122C442290E835E0FC90EF
:1032BA0038B8230493C0E0EC2393C0E022903BA6E5
:1032CA00122C2E903A65122C2E90E835E0F89038A0
:1032DA00D37C00E4A39370030C80F8ECB500F412DD
:1032EA002C077429122C3374D3122C44122BF21289
:1032FA00311E9036141231C222903BA6122C2E9007
:10330A003A71122C2E74C9122C441232B4903674AB
:10331A001231C222903A7C122C2E903AA5122C2EEF
:10332A00E57612347274C4122C44E576122C7FE5C9
:10333A0076120A797490122C44122BF290E837E430
:10334A00F090E836E4F090E838E576F090335D12D4
:10335A0031C22290E837E0FFBE0F080FBF110D7F80
:10336A00008009BE0E221FBFFF027F1090E837EFD0
:10337A00F070097490122C44740D800724C3122C27
:10338A0044740E90F800F022EF7036BE0B0A123326
:10339A00FB04B50010E4800DBE0C5E1233FB14B4BE
:1033AA00FF03E50014F090E838E0FF12347274C4A9
:1033BA00122C44EF122C7F7490122C44EF120A79CB
:1033CA0022BE0B0B123CD904B47E107420800CBEB2
:1033DA000C27123CD914B41F02747DF0F8122BF991
:1033EA00E8122C33EF24C3122C44740E90F800F028
:1033FA0022A8770890E838E022BE0A13122BF97443
:10340A0080122C447C149039C5122C4B02369CBE77
:10341A000D1990E837E06013123CF690E837E4F0B3
:10342A007490122C44740D90F800F022903A7C1299
:10343A002C2E903A8F122C2EE576123472120F83AC
:10344A0012347F120F831234987490122C44122B68
:10345A00F290E837E4F090E836E4F090E838E57660
:10346A00F09034C61231C222C0E07491122C44D0BA
:10347A00E01236D622780E540F14F5F074C3122CCB
:10348A00441235C71235F290E839E5F0F022F854C3
:10349A000FB40400400824FDF5F07803800CE8C45A
:1034AA00540F90370693F5F0780474CA122C44121C
:1034BA0035C71235F290E83AE5F0F02290E837E0A5
:1034CA00FFBE0F080FBF030D7F008009BE0E381F15
:1034DA00BFFF027F02BF020990E839E0B40300503F
:1034EA00E090E837EFF0122BF9903D2BE493600B54
:1034FA00122C44741D122C33A380F1903D2BEF93B0
:03350A00122C443C
:10350D00122BF222BE0B0A123D2F04B50010E480DF
:10351D000DBE0C4B123D2F14B4FF03E50014A98210
:10352D00B9380AC0E0123594D0E090E838F090E850
:10353D0038E012347290E837E0700E90E838E0759C
:10354D0083EA4400F582E080031235A2C0E0123414
:10355D007FD0E012349890E837E0FF12350522BE97
:10356D000A1C90E837E07003123594122BF9748021
:10357D00122C447C149039B1122C4B02369CBE0D8A
:10358D00DD90E837E0D2541235A2FB90E838E0FE2A
:10359D00C24A02248590E839E09035B093B44400D6
:1035AD004006220102034455F890E83AE09037D7DF
:1035BD009354F0482290E835E0F8903911E8939053
:1035CD00E830F0903920E89390E831F090392FE809
:1035DD00230493F9E8239390E833F0A3E9F02290C4
:1035ED00E832E0F5F090E830E0FCC0F0A4D0F0F95E
:1035FD0090E830E0FC90E833E0F8A3E029F582E4B0
:10360D0038F583122C4B22A81FBE0A00500F75A04F
:10361D00E8EEF208B83F131818F208800DBE0E023E
:10362D008003BE0F3218B83A0108881F7491203EEE
:10363D000274D1122C4412312D400A903BA77C0309
:10364D00122C4B8007D256121FD5C2567493203EB2
:10365D000274D3122C4422BE0A028033BE0DF7121F
:10366D00312D403E02386D90E831E0F890E832E0BF
:10367D00BE0B0704B5000CE48009BE0C0F14B4FF9B
:10368D0002E814F074C9122C441235ECBE0A1090E5
:10369D003C2A122C2E122BF99031D11231C222BE9E
:1036AD000D1B90E835E0F8B400028002D25490383A
:1036BD009C93E8230493C0E0E82393C0E022E4A2A6
:1036CD003892E0FC02376AE5772401FDE43400FA14
:1036DD00023776E55F540FB402057C0002376AB4F9
:1036ED0004047C018077B405F17C028070E55FC431
:1036FD00540790370693FC8064000001030002908C
:10370D00E86EE0FD90E86CE0FA53020F805B90E903
:10371D0004E0FC804890E86AE0FD90E868E0FA5328
:10372D00020F804590E863E0F4541FFD7A00D21E2D
:10373D00803790E863E0F4546003C4FC801F90E987
:10374D0030E0FD7A00D21E802090E866E0FD7A0020
:10375D00D21E801590ED00E0FD7A00800C1235C26E
:10376D0090E832ECF01235EC22D256121FD5C2562B
:10377D00C21E2290E832E0A2E09238023867123180
:10378D005440046002F57702386790E832E09037D4
:10379D00BD93F9540FB40209E55F540FB40202A9A9
:1037AD005F895FC00012062912072DD0000238670D
:1037BD0012445590E832E09037D793F55FF9895F61
:1037CD00C00012072DD0000238671222523290E845
:1037DD0055E090E86CF0A3F090E854E090E86EF0BE
:1037ED00A3F0807690E832E090E904F0806C90E8E8
:0137FD005576
:1037FE00E090E868F0A3F090E854E090E86AF0A357
:10380E00F0805690E854E0F4541FFC90E863E054C6
:10381E00604CF0804490E832E0F4540323C4FC90F2
:10382E00E863E0541F4CF0803090E854E090E930AB
:10383E00F0802690E854E090E866540FF0801A90DD
:10384E00E854E090ED00F0FEC000E41221B17403E4
:10385E001221B1EE1221B1D0001232AB1232B412DB
:10386E002BF9903C2A122C2E9031D11231C22222E9
:10387E00330332C73303330333033436331E32C7B5
:10388E0032C732C732C732C7330332C732C7378067
:10389E0037DB37F1379737C0387D387D378B383780
:1038AE00384137FB38113823384D36CB370C371BA0
:1038BE0036E036FA387D387D36D4374B37563722D8
:1038CE003731373F376100312D393939000000006B
:1038DE000000322D32353600312D313600312D318A
:1038EE003600312D39393900322D33300000302D6C
:1038FE00323535008B8C8F8A87D4D48F91919192EB
:10390E008A91D40300030A0A000000000000000799
:10391E000003020002030400000000000000040087
:10392E00053B0700003B013ABB3AD90000000000FE
:10393E000000000000000000003B0D00003B29537A
:10394E0063616E206D6F64651D2020202020202075
:10395E002020205363616E2074696D651D20202028
:10396E0020202020202020506F776572206F6E203F
:10397E007363616E1D2020202020204B6579626FBD
:10398E006172641D20202020202020202020204D28
:10399E006F7573651D2020202020202020202020E0
:1039AE00202020435055206B6579626F6172642F21
:1039BE006D6F7573652020435055206E616D657374
:1039CE0020202020202020202020204D6178696D8D
:1039DE00756D20706F7274731D202020202020457D
:1039EE007870616E73696F6E2077696474681D20DC
:1039FE00202020457870616E73696F6E20756E6938
:103A0E0074731D20202020566964656F20626C61DE
:103A1E006E6B2074696D651D2020204B42207261F3
:103A2E007465206B6579732F7365631D2020204BA1
:103A3E00422064656C61791D2020202020202020EA
:103A4E0020202053756E206B62206C616E6775614D
:103A5E0067651D20202020C04E65772076616C752D
:103A6E00652800C043686F6F73659E9F200080437A
:103A7E00686F6F7365209E9F7F7E20204350551D7B
:103A8E0000C04B421D202020204D531D2020202001
:103A9E0020202020202000C04E616D652020202097
:103AAE0020202020202020202020202000504320D5
:103ABE00202020202020204D616320202020202047
:103ACE002053756E2020202020202050532F32208E
:103ADE0020202020205365724D6963736F667453E6
:103AEE00657250436D6F757365536572204F7468C0
:033AFE00657220CE
:103B01004E6F205965734F66664F6E20536C6F7709
:103B11002020204D656469756D20466173742020F5
:103B2100204661737465737450433150433250437E
:103B3100334D616353756E8052657365742073757F
:103B4100636365737366756C2020202000C048692B
:103B51007420656E74657220746F2070726F636576
:103B6100656400805265736574206661696C656483
:103B710020202020202020200080436F6E6669676E
:103B810075726174696F6E2072657365742000804F
:103B9100436F6E66696775726174696F6E206261E9
:103BA1006420202000C02020202020202020202050
:103BB10020202020202020202020008020202020C4
:103BC10020202020202020202020202020202020F4
:103BD10000C050726F6772616D20636F7272757091
:103BE10074656420202000C0536C617665206C6987
:103BF1006E6B2062616420202020202000C053745D
:103C0100617475731D206E6F726D616C20202020B0
:103C1100202000C05374617475731D206E6F206382
:103C2100707520706F77657200C0456E746572A5FE
:103C310073656C656374209E9FA56974656D0080D2
:103C41005361766520636F6E666967757261746929
:103C51006F6E202000C0456E7465722063686F69C5
:103C610063659E9F20596573202000CF59657300BD
:103C7100CF4E6F2000805363616E206D6F646520AD
:103C810020202020202020202020004E616D650072
:103C9100203D2000204368616E676520592F4E2F1B
:103CA1004553433F20004F6E204F6666C0537461F9
:103CB1007475731D206E6F742073656C6563746514
:103CC1006400C05374617475731D20766964656FF7
:103CD100206F66662020200090E838E05403C4F885
:103CE10090E837E014540F42007583EB7400543FA1
:103CF10048F582E02212093390E838E0120A6A534B
:103D010082C075A0EB79001214D92278007900D90C
:103D1100FED8FC2290E837E4F0FF123D1F22903DCF
:103D21002BEF93122C44122BF22290C2C900BF0137
:103D310007780590E839E022780490E83A5006A81F
:103D4100770890E838E022E575C4540F4410F582F5
:103D51007583E9E022C0E0740925748355D8D360E6
:103D610001C3D0E0220201080444B1C0B3B4B5B725
:103D710040B9B0B8BB413A424330313233343536C1
:103D8100373839BF3FC13BC2C3B2E1E2E3E4E5E604
:103D9100E7E8E9EAEBECEDEEEFF0F1F2F3F4F5F63A
:103DA100F7F8F9FA3C3E3DB6BA2F61626364656685
:103DB1006768696A6B6C6D6E6F707172737475761A
:103DC1007778797ABCBEBDAF1B6030313233343580
:103DD100363738392D3D5B5D5C3B272C2E2F200873
:103DE100090D1B7E2921402324255E262A285F2BCD
:043DF1007B7D7C3A20
:103DF500223C3E3F2008090D2030322F31322F3929
:103E05003820436F707972696768742031393930A9
:103E15002D3139393820526F736520456C656374CF
:103E2500726F6E69637320C2A91290A775F02C1288
:103E35003F0B123F2C123F5120083F123ED8403A0B
:103E4500D20ED279A950A7060953016FA707B7FF6C
:103E550002800EB7B607E506B4B602800409530121
:103E65006F89503001147420128552744B1285529B
:103E7500E506128534E5071285341290B41289F2ED
:103E8500D2A922128A1DC2A91290A775F03C123F31
:103E95000B123F2C123F51200830123ED8402BD236
:103EA5000DD279A959A7060953014FA7070953014F
:103EB5004F8959300114744D128552E50612853427
:103EC500E50712853474201285521290B41289F2D6
:103ED500D2A922123F61402D7D08123F6140263054
:103EE5000903C38001D3E50633F506DDED7D081230
:103EF5003F614011300903C38001D3E50733F5075E
:103F0500DDED123F612253B0CB7C92000000DCFB5B
:103F150043B0347C1ADCFEE5F07D0833123FAF0078
:103F250000000000DDF52253B0CB7C1FDCFE43B062
:103F3500347C0DDCFE20B4028004C208800D7CFFB9
:103F450020B406DCFBD2088002C20822C2087C3FEE
:103F550030B406DCFBD2088002C208227CFFDC02FA
:103F6500801D20B4F97C000C30B4FCC3EC940E50D9
:103F75000AC3EC94034008C2098002D209C322D3C4
:103F8500227C26DCFE227D10C5F0D3123FAF000057
:103F9500000000000033123FAFBD0904C5F08003E7
:103FA500000000DDF0C3123FAF22C0E053B0CB7C70
:103FB5000D500280027C1BDCFE43B0347C135002A2
:103FC50080027C05DCFED0E0227C127DFFDDFEDC7C
:103FD500FA22128A1DC2A91290A775F02B123F0B67
:103FE500123F2C123F8675F06275E003123F8B126B
:103FF50090B41289F2D2A9224300F830E0055300AB
:10400500FB800343000430E1055300FE80034300B9
:104015000130E2055300FD8003430002E500221252
:104025003FFD85E0827583FF128A1DC2A91290A704
:1040350075F02A123F0B123F2C123F868582E085D0
:0E40450083F0123F8BC20C1290B4D2A922223B
:1040530002972B32FFFFFFFFFFFFFF758C10D26B20
:10406300327583F011607583F411601286997900BB
:104073007583E8E92480F582E07583EAF582E0122E
:1040830080B709B904EA90F400786675F000E55F3B
:104093005407117990F410117990F408787775F03A
:1040A30003117990F41A7415F07582187403F022D1
:1040B30075821274C0F075820FE075821FE07582FD
:1040C300047470F0758214F022438202741AF0F0C3
:1040D3005382F8438200741330F2027407A2F09201
:1040E300E0F07407F05382F8438201E8F05382F85A
:1040F300438202748020F1027490F074A020F102D4
:1041030074B0F07405F022C4540F75F0007866B4EF
:104113000500401AB4050575F0018012B406077551
:10412300F00578668008B407F375F0017899758314
:10413300F0E9C403F58212807922E590543C537D63
:10414300C3427D227583F030E3037583F4C40324F3
:1041530001F582E030E20D5382F8438203E8F01266
:104163008EF7C322D3755D0022E8B57800401B901B
:10417300928193FE55906004EE427D22EE557D6060
:1041830009E8784D11F4EEF4527D22F9E574917B40
:1041930074EF91A4E574917BE991A42279387B3083
:1041A300D255E95403C074F574B120D07450028021
:1041B30053E578601BE95403F8B578005002803466
:1041C30090E930E08578F0A428C39578F5828007DC
:1041D300E954032400F5827583EAE05407B4070524
:1041E300128356801FB40402801A40045195801430
:1041F300E0C45407D1CA430104D1CA5301FBE954B3
:1042030003F83119090B309803128A58B93C93C249
:104213005522128E66128520204E49404720020304
:1042230020182BE5795407B40707E5741280F4804E
:104233002AB4041175F0FF128F3250280554E55447
:10424300B40A2A801F4007E57412858F8016E5742F
:1042530012847BE890E885F01284B550070554E595
:1042630054B4A00975540005551553C322D3221223
:104273008520204E685002806420020320183DE50B
:1042830079C45407B4041888F009E3F8128F49502D
:104293000A055DE55DB40A4C755D00755C0022405E
:1042A30011B40707E5741285FF8032E5741280F4B8
:1042B3008022B40207E5741280F48018E5749092AA
:1042C3008593557D6017E574D2E212847BE81284EE
:1042D300B5500A225007055DE55DB4A007755D0082
:1042E300055E155C22E754036002801AE954031249
:1042F30083A0400122B71005770051B822B40139D9
:1043030077037E0051B880737583E9E95403F84459
:1043130010F582EEA2E292F0A2E092F1A2E392F211
:10432300A2E192F3E5F0540FF0E576200205E5757E
:10433300C4540FB50044D25C22B40E067710128920
:014343004930
:1043440022B40F0477068032B402028010B4030250
:10435400800BB40A028006B40B02800122E95403E4
:10436400F8E576200205E575C4540FB5000B90E816
:10437400402582F582EEF0D27522E790972293B41D
:10438400040E90ED00E0A2E77404500D740380095C
:10439400B45A0690ED00E0547FF8E9540312858F77
:1043A400171289492290F41112838950117420B193
:1043B40052746BB152E8B13490F00112839690F0CC
:1043C4000112838950117420B1527463B152E8B15F
:1043D4003490F40112839622E020E002C322438247
:1043E40003E0F8D322E030E2FC438203E8F02275D4
:1043F40083F0F830E3037583F4C4032401F582E009
:1044040020E004C3E4800B5382F8438203E0128E5D
:10441400FCD3FE22A2E2924AC0E0917BD0E0540396
:104424009084A093C002FA128A1D7C0878009144FB
:10443400E5C8304A02E5C05AC36001D3EE13FEDC7E
:10444400ED9144E5C8304A02E5C05A60010C91443C
:10445400E5C8304A02E5C05AC24A6002D24AC39152
:1044640026E572F442C8E573F442C01289F2D00220
:10447400ECA2E0EE22C0E0400AE57252C8E57352B5
:10448400C0800AE572F442C8E573F442C0D0E07F0C
:104494000180027F04DFFEC0E0E57052C8E571527E
:1044A400C07F0EDFFEE570F442C8E571F442C0D26D
:1044B40065E570F4600855C88009C0E080F1E571D5
:1044C400F455C07002C265D0E022FE2055043019B4
:1044D4000122A2E2C2E290849C937FFF4001CFF5C7
:1044E4007103F573CFF57003F57222F7FDDF7F04D6
:1044F4000110407D00C0E0128F101284CBD0E05038
:1045040002DDF222205506301903022130BE0400D8
:104514005005128ED48003128EE8FFEEA2E2C2E2AE
:1045240090851C93400445C8800245C0CFBFFF025C
:104534008002D322128A1D12846B30651EC312843A
:1045440026306517A2D0B37C091312842630650B7C
:10455400DCF7D3128426C31289F222D3FCE572F469
:1045640042C8E573F442C0ECD380ECF3FCCF3FC007
:10457400E0740925748355D8D36001C3D0E02202C6
:10458400010804300111C0E0C4540FB149D0E0C0A7
:10459400E0540FB149D0E022B40A004002240724B9
:1045A40030300107F5993099FDC2992290E857E01F
:1045B400D5E0027406F0B406247938E7B41002801A
:1045C400045403600FB24020400A77005301F77788
:1045D40000430108E52803F52809B940DE22C81282
:1045E4008F01C890970993FAC3B1A87C08E813B166
:1045F400A8DCFBD3B1A822CA858AF020F7FA858A01
:10460400F030F7FA400452C88004F442C8F480241D
:10461400C8128F06C8C3B1D57C08E813B1D5DCFB3A
:10462400D3B1D522CA858AF020F7FA858AF030F70B
:01463400FA8B
:10463500B392B2858AF020F7FA858AF030F7FA85C9
:104645008AF020F7FA858AF030F7FACA22C8128F65
:1046550001C890970993FAC3D11C7C09E8A2D0B38D
:1046650013D11CDCFBD3D11CC322CA858AF020F5EB
:10467500FA858AF030F5FA4006F442C8F480025211
:10468500C8858AF020F5FA858AF030F5FA858AF032
:1046950020F5FA858AF030F5FACA22AC7420020CAE
:1046A500E57554C07023E575C45403FC74382CF8C3
:1046B5002404F9E6B41001225403700FE7B4100185
:1046C50022B434012254037002D322C322C3200230
:1046D5000DE57554C0700EE575C454038002E5768A
:1046E500B50402D322C3227C0075A0E87880EC20B3
:1046F500021F12867F401890E930E0F5F0ECB5789E
:10470500005003A4800BE578A42CC395788002E5BE
:1047150076F2080CBC04D722E954039084A093FADE
:10472500E9A2E2E5C85002E5C0FE5A7044EE035A1C
:10473500603F5012E5C8FE5A7007EE035A700280BA
:1047450030E5C05A702BE9540771C5304A0F20D0A7
:10475500045004800A50087433C24A80027422B996
:104765003C005005128ED98003128EED304A02802E
:10477500030287A3E7B4100AE920E22CBEFF320248
:1047850087DDE930E2F912874FB4EEF3BEEC0302A0
:1047950087DDBEFF030287DDAC060287F754039071
:1047A500E87C2582F582E02212874FB4F303128953
:1047B50058770DE920E23A540390E840FC2582F54C
:1047C50082E0B4ED1FEE7583E98C82438210F0D14F
:1047D5007F501EE07583E98C82438210F0D25C0223
:1047E50088338047B4F00ABE000A540323232416F5
:1047F500F70288D71289375407B40400501BEE30EE
:10480500020D30E70AA2E45403B392E4F0800AE013
:1048150054F05306034EC2E7F0D17F5064EEA2E791
:104825009207C2E7E0F579D25D80569091FF7C252D
:10483500B93C0040059092237C45A3A3ECB5824486
:10484500B445077CFEE954078012BEFE19E95403FE
:104855007CFAB5740790E885ECF0E57412847BEC7E
:104865001284B50288D775A0E8E954032440F8E21C
:10487500F87429B8FE005014B8FB00400F740D778A
:104885000D0288D7E493B506B1A3E493F7E954077D
:104895001288A3E9540730E26BC2E2B57400BEF298
:1048A5000C12893754F07002773A0288D7D2E2BEEB
:1048B500E91C750504F500E812847BE505240983E8
:1048C5001284B540F2D505EF805B3C0310FA909257
:1048D50085540393BEF404427D804ABEF50B20182F
:1048E500F82019F5F4527D803CBEFFED1289AB80AE
:1048F500EDA2E2C2E290E840500390E87C2582F503
:1049050082EEF022BEFF1E7583E9E95403F582436A
:104915008210E4F012893754F04402F0E95403FCA4
:0349250012867F78
:10492800925CE7B434028004540360558B0006E6B9
:10493800FEE7B4080050079091BB936E7043E9A25C
:10494800E2E5C85002E5C0035A7003168033E95403
:1049580003C074F574128520D0744025E9540712F9
:10496800847BE79091C393FCE95407B5740590E8FC
:1049780085ECF0EC1284B5500316800517760031EB
:1049880049227583E8E954032480F582E07583EAB7
:10499800F582E022E924CB83522822FEFDFBF7EFC3
:1049A800DFBF7FBEC8028038BE640812899BB4C8C6
:1049B8002D802DBE502812899BB46422C3C0D0120A
:1049C8008937D0D0540F50024410FEE95403B5780B
:1049D80000400BCEF0CEFC12867F50028E797E000E
:1049E8001289A0EEF0221289A0E02290E878E9541A
:1049F800032582F58222C006D31289727E001289AD
:104A080095D00622201835201932128520204E2CE8
:104A1800402AE579B4440975F0FF78B6128F32223E
:104A2800B4550FE574780D12858FE574788D12856D
:104A38008F22B47707E57478B31280F42220022518
:104A480030AF24C0E0203B12E55F64446015E55FA9
:104A58006455600FC289D2A8D2B2203A06C28BD25E
:104A6800AAD2B3D0E0D2A92220023530AF3430A880
:104A780016202FFD203B10C2A87CFF20B204DCFBCF
:104A8800D266C2B275250830AA162037FD203A1022
:104A9800C2AA7CFF20B304DCFBD267C2B375260828
:104AA800C2A922200236205E33205930205A2D20F8
:104AB800582A203D27205C24205D21203C1E205BB5
:104AC8001BC3E5592410955A540FB40900500DE53D
:104AD80099C298201207B43F0485769922F5993037
:104AE80099FDC29910124C205E48B40005D212C23A
:104AF8002022B40105D212D22022F890E852E0C850
:104B0800B40D1518E577B50000400A8876C270C262
:104B180038D26FD215E4F02224D0B40A005013C85A
:104B2800C0F075F00AA4D0F030D2028005285001F8
:104B3800E4F02220200AA850F60853006F8850227B
:104B4800A859F60853004F8859D24922855600754E
:104B58005300E579540FFE300205200705800C301C
:104B680018097E03B4030050027E0275A0E879207C
:104B7800BE0402801FB81A028003B89A17EE1423E5
:104B880023FE909245755300EE936007F3090E05D6
:104B98005380F522E86007A2E792F0028B97BE03E4
:104BA80003028BDF4011E557A2E792F0C2E7B41980
:104BB8000040EEF8028C1EE557B4050050E374E09F
:104BC800F309755301E5571423255714F890926596
:104BD800BE0103909259E89360070553F3A3098037
:104BE800F522BE0133E8547FB40F0C30F002803A4E
:104BF800909271780080DF91466009A2F092E7F305
:104C08007553012290928974E0F309E8547F93A2C6
:014C1800F0AB
:104C190092E7F375530222BE0247E8547FB41F039B
:104C2900301806B40F0E30F00475530022909278B4
:104C3900780080A19146600F75530130F00674F039
:104C49000553F309E8F32290930975530274E0F3CD
:104C59000930F00974F00553F30953007FE893F321
:104C690022BE0304914680D0BE0404916E8003BE27
:104C7900051DE5567014B81905BE04AD8003BE05BF
:104C8900A89096F4E8C2E79361B0914661B02222F8
:104C9900EE14909389C0F075F080A42489F582E51B
:104CA900F0D0F03493F583E8C2E793B4FF06D0E07F
:104CB900D0E061DF6001F822B81A03D38004B89A02
:104CC90009C3D18F92E2F0D25C22B87C16D18FD27F
:104CD9005CB2E2F0D2F078FC30E207C2F0787C7581
:104CE900530122B8FC06D0E0D0E061DFB87B06D1E1
:104CF9008FB2E18007B80E07D18FB2E0D25CF02203
:104D0900D27375A0E87928E579C4540720192B20B6
:104D19001823B40706D104755C0322B4040691F381
:104D2900755C02224006B11D755C0522B40206B10C
:104D3900C0755C03226003B17B22B17F2290E82D0C
:104D4900E0F5F0A3E0A2F492E6D2E790E829F0902A
:104D5900E82FE0A2F592E7F404A2E792E6A2F0B305
:104D690092E790E828F02290E82DE0F875F080F4B9
:104D7900A2E092F2A2E192F0A2E292F1E5F090E8CB
:104D890028F088F0A2F490E82EE090E829B151A229
:104D9900F590E82FE090E82AB15122401420E70469
:104DA9007800801B04F853007F7002787F747F803D
:104DB9000EB48000400478008005D2E7F87480F0D2
:104DC900A3A3E8F022740380027404FCF55C90E864
:104DD9002D75A0E87828E0F208A3DCFA22A85A90F9
:104DE900E82D7C03E6F008A353004FDCF7200211FD
:104DF900303908E57954F060088003204D03E480D8
:104E090002E608F053004F885A2290E82DE075F029
:104E190040A2E092F5A2E192F4A2E492F1A2E59215
:104E2900F390E82EE0A2E692F0543F90E829F09042
:104E3900E82FE0A2F392E7F404A2E692F2A2E79245
:104E4900F3543F90E82AF090E828E5F0F02290E842
:104E59002DE075F090A2E092F2A2E292F1A2E19225
:104E6900F0A2E4B392F4A2E5B392F390E82EE070D5
:104E790002D2F430E702F40490E829F090E82FE038
:104E89007002D2F330E702F40490E82AF090E8289F
:104E9900E5F0F022201918201815E57954F0700F63
:104EA900755C02755E2890E82874AAF0A3E4F022E4
:104EB900E5795407B40404747F800440177430689A
:104EC900A2E7C2E7700EE574908E8B934004F4520A
:104ED900C02242C02208022080E576200205E5753D
:104EE900C4540F4410F5827583E9E022751E74805D
:104EF90076751E738071751E53806C751E6D806783
:034F0900751E2AE8
:104F0C008062751E2B805D751E798058751E7A80A7
:104F1C0053751E6B804E751E4B8049751E63804405
:104F2C00751E43803F751E78803A751E5880357506
:104F3C001E708030751E50802B751E758026751E58
:104F4C00718021751E51801C751E628017751E4262
:104F5C008012751E72800D751E778008751E6D800F
:104F6C0003751E6E300111C0E07420128552E51ECF
:104F7C00128552D0E012853422C20DD20E30010CB3
:104F8C00C8128F15C8C5F0128F15C5F012910822E2
:104F9C00D20DC20E30010CC8128F1AC8C5F0128F78
:104FAC001AC5F012910822C20843C83E7C0FDC02DD
:104FBC00804D7DFFE5C8553C6004DDF880F07C0039
:104FCC000C0000E5C8553C60F7C3EC9467500A2010
:104FDC00082D1291B2D20880D07C000CE5C8553C4B
:104FEC0070F9C3EC9409500280157D0812907C4036
:104FFC000E300903C38001D3E833F8DDEFC322D3AD
:10500C0022300A16E53F52C8E53D52C07C68DCFEF2
:10501C00E53C42C0E53E42C8C20A2200E8B42A067A
:10502C00D20BD20C804FC20BE854F3B42009300ED3
:10503C003EC20ED20F803AE854F3B43009300D2F33
:10504C00C20DD20F802BE854F3B4220A8EF08FE0FD
:10505C00C20ED20F801B8017E8B42F0C75F063754D
:10506C00E002C20ED20F8009E8540FB40B0100C24B
:10507C000F7C5FDCFE227D10C5F0D3129053000034
:10508C00000000000033129053BD0904C5F08003EA
:10509C00000000DDF0C312905322C0E0E53F52C87F
:1050AC00E53D52C07C0B500280027C19DCFEE53CD5
:1050BC0042C0E53E42C87C13500280027C06DCFEF6
:1050CC00D0E0227CFFDC028023E5C8553C70F67CE6
:1050DC00000CE5C8553C60F9C3EC9408500AC3ECCD
:1050EC0094044008C2098002D209C322D322853C11
:1050FC001E853D1D853E1C853F1B22851E3C851D46
:10510C003D851C3E851B3F227C26DCFE80151290C3
:10511C007CC2087CFFE5C8553C6006DCF8D20880F0
:10512C0002C2082212907C40257D0812907C300926
:10513C0003C38001D3EE33FEDDF17D0812907C3089
:10514C000903C38001D3EF33FFDDF112907C228879
:10515C008285F083128A1D1290A7129189128F609A
:10516C00402F129151300A028002800B128FBA85A7
:10517C0082E08583F080E6128FD4200B0E300F1165
:10518C008582E08583F012902F80061290C11290D8
:10519C00DD1290B41289F222200D028003200E2D14
:1051AC00E854F0B400028021E854F0B42010E8B4C4
:1051BC002E03029186E8B42A028012200D0BE854CB
:1051CC00F0B43009200E028004D20A8002C20A22F6
:1051DC00C082C083E5749091AA93F53C64FFF53DC1
:1051EC00E5749091AE93F53E64FFF53FD083D08289
:0151FC002290
:1051FD00040110400C0330C07C047DC8DDFEDCFAD8
:10520D0022000A01000001030100AAFA000000AA11
:10521D00FA0083ABFA00FA000000FA00000000FA71
:10522D00000001FA000002FA000003FA0000EE008F
:10523D000000FE000000BFB0FA00000008FA0000F8
:10524D00000003FA0000FCFF02F20BED11F311F464
:10525D000DF011F50DF60DF70DF80DF90DFA0DFB1D
:10526D000DFC0DFD0DEE25D229EF2FFF07F60DF5E7
:10527D000DF40DF311F216E811E70DE60DEA0DE947
:10528D0000EC0DF00DEE0DEB34E43D3ABA00005894
:10529D00F0580014F014000000000077F77F002A8A
:1052AD000000360000AA0000B600001200005900F0
:1052BD0000F01200F05900E11D45E19DC500E1141B
:1052CD0077E1F014F077000408102001024080000F
:1052DD00000000000000000000000000370000008A
:1052ED000000000000000000000000005D00000054
:1052FD0000000000000000000000000000000000A1
:10530D000000000000000000000000000000000090
:10531D00000000000000000000001D00385B5C5222
:10532D0053474F495148504B4D00350000001C006C
:10533D000000000000000000000000000000000060
:10534D00000000000000000000000000004600000A
:10535D000000000000000000000000007C000000C4
:10536D000000000000000000000000002F00000001
:10537D000000000000000000000000000000000020
:10538D000000000000000000000000000000000010
:10539D00000000000000000000001400111F277025
:1053AD00716C697D7A75726B74004A0000005A0049
:1053BD0000000000000000000000000000000000E0
:1053CD00000000000000000000000000007E000052
:1053DD003B3C3D3E3F404142434457580046FF52FF
:1053ED004F50514B4C4D474849FFFF5600FFFF2B87
:1053FD00FFFFFFFFFFFFFFFFFFFFFFFFFF01290B78
:10540D0002030405060708090A0C0D1A1B2B272891
:10541D00333435390E0F1C2A361D003800000000BC
:10542D00000000000000000000FF00374A4E00534E
:10543D001E302E2012212223172425263231181931
:10544D0010131F14162F112D152C453A5400FF0063
:10545D000506040C030B830A01097807007EFF7013
:10546D0069727A6B73746C757DFF60610062625D49
:10547D00FFFFFFFFFFFFFFFFFFFFFFFFFF760E4563
:10548D00161E26252E363D3E464E55545B5D4C521E
:10549D0041494A29660D5A125914001100000000A5
:1054AD00000000000000000000FF007C7B7900710F
:1054BD001C322123242B3433433B424B3A31444D90
:1054CD00152D1B2C3C2A1D22351A77588400FF0000
:1054DD00070F171F272F373F474F565E575F6270D5
:0F54ED0069727A6B73746C757DFF80138D81818A
:1054FC0053FFFFFFFFFFFFFFFFFFFF80FFFF080EC3
:10550C0045161E26252E363D3E464E55545B5C4CAC
:10551C005241494A29660D5A1259115819398B8C26
:10552C0067646E656F6D6360616AFF777E847C79FA
:10553C00711C322123242B3433433B424B3A3144EC
:10554C004D152D1B2C3C2A1D22351A7614FFFFFFFE
:10555C00007A78637660616264656D676F696B7100
:10556C0052535455565758595B5C39370A7F7F7FD5
:10557C002AFFFFFFFFFFFFFFFFFFFFFFFFFF35329B
:10558C001D1213141517161A1C191B18211E2A2963
:10559C00272B2F2C31333024387B367D3A7C373710
:1055AC007275737774793E3D3B3C514B434E454C81
:1055BC0041000B08020E030504222628252E2D1F60
:1055CC00230C0F011120090D0710064739FFFF3975
:1055DC00000506080A0C0E10111207090B161715F8
:1055EC005E7071725B5C5D444546FFFF7C30303011
:1055FC0058FFFFFFFFFFFFFFFFFFFFFFFF7F1D2A8D
:10560C00271E1F20212223242526282940415856B5
:10561C00576B6C6D792B3559636E4C43130D787A3F
:10562C002C42344A607B141B181CFF2E2F477D5ACA
:10563C00324D68664F385051523D5354556A693E4D
:10564C003F36394E3A3C6737653B646277FFFFFF64
:10565C00FF565758595A5B5C5D5E5F6061626364CC
:10566C003A393F403E444542434AFFFFFFFFFFFFAC
:10567C00FFFFFFFFFFFFFFFFFFFFFFFFFFFF0636F0
:10568C002D070D0E15161D1E25262E353037382AE2
:10569C00312C3334523C0832050402555354FFFF6D
:1056AC00653D666867695049484FFF6B6C4B6D519F
:1056BC00410A231B111012191A272122292B2428E5
:1056CC002F09170B18201C0F141F136A03FFFFFF61
:1056DC0000565758595A646566676871728182839F
:1056EC0092969798999A9B9D9E9FFFFFFFFFFFFFB5
:1056FC0073747C7D80A0FFFFFFFFFFFFFFFFBFC91E
:10570C00EFC0C5CBD0D6DBE0E5EAF9F5FAF6F7F257
:10571C00FBE8EDF3D4BCBEBDAEABAFADACB2B1FFEC
:10572C00888C8A8D8E8FAAA9A7A8FFA2A3A4E8951E
:10573C0094C2D9CECDCCD2D8DDE6E2E7ECE3DEEBF9
:10574C00F0C1D1C7D7E1D3C6C8DCC3A1B0FFFFFFFE
:10575C00FBFEEFBF51762D02040103191A313348B9
:10576C00495F61300F7374757F007F04FF005AFE30
:10577C00000075B0FF75810775E80475D8DF75906A
:10578C00FCE4787FF6D8FDE590F454C02440F57F16
:10579C0060FE74FFF57575506075516075594075F4
:1057AC005A40757B00757C0090E8577406F0D20265
:1057BC00129B86B4E6FA129B86FC90ED00129B8637
:1057CC00F0A3DCF9E57FC4FE90E9107C04129B8603
:1057DC00602AFF540CD2F0B50602C2F0129B862050
:0257EC00F0EBE0
:1057EE00F0A3DCE77C04EFC4540FB4000590E9206D
:1057FE0080D9B401D690EA0080D11280111280EACD
:10580E005389F0438901D28CD2A9D2AF437DC330E4
:10581E006B03129B22306D09E55C7005128E4AC235
:10582E006D12864D4003029AD8E57BB57C02802727
:10583E0075A0E8A87CE2F9E57412847BE91284B5C0
:10584E00500A0554E554B4A00975540008B8100266
:10585E007800887C029A4F75A0F47819E220E00354
:10586E00029953781B20E564E270030298C8B4FFD6
:10587E0022129914307BE910E612A95077000953D1
:10588E00016FF70953016F895002994EF57EC224BC
:10589E00029928307BCAF5F054FCB42822129914D0
:1058AE00F975A0E8A87B30F10574E012990C30F080
:1058BE000574F012990CE912990C887B02994EA985
:1058CE0050A7F00953016F895002994E7C04A959D3
:1058DE00781BE2FE307B33C3E5592410955A540FE2
:1058EE00B40C00748040027481129B6FB4801BEE66
:1058FE0080097819E230E0FC781BE2128534F70952
:10590E0053014FDCED895902994E029953129914A5
:10591E00A2E792235000F57E537E7FC224547FB4BB
:10592E0001028013B43002800EB403028009F853D2
:10593E0000F0B84015D2767819E230E0FC30E5037D
:10594E00029887781BE2F57AD224202320D27C801D
:10595E0047F208B810027800227819E230E0FC20F5
:10596E00E504781BE222D0E0D0E0029887307B2855
:10597E0075A0E8A87B74EF12990CE57E12990C3095
:10598E00240F307607C27674EF12990CE57A1299CD
:10599E000C887B7480129B6F107C03029A4FE57EFD
:1059AE00B4012FC207E57AFE54F0B50614E57F6EFA
:1059BE0054C0700DEEF5755430C4F576D26F029A60
:1059CE004AC27B7575FF7576FF74AA42C0C2EC029F
:1059DE009A4FB4160C7440B57FE77480129B6F809B
:1059EE00E0B40309E57A90ED00F0029A4FB4301955
:1059FE00E57AC454C0B57F0EE57A54039092859330
:105A0E00457DC57DD26D029A47F95301F0B9402408
:105A1E00F9C4657F54C0701AE95403F9307B06B59A
:105A2E007403857A797583EA4400F582E57AF0127B
:105A3E0080B78058B40924207B028050128E8FF8D4
:105A4E00129B17540FC44200C074857674128520C1
:105A5E00D074B3E892E7129B6F8039B40C07307B99
:105A6E0002D2EC8027B40208C2EC74AA42C0801C99
:105A7E00B43119307B14E579540FB40400500BE5A2
:105A8E0074D2E212847BE41284B58000307B0574FC
:105A9E0080129B6F306F24E55C6015207209D27204
:105AAE0090E83FE4F0801490E83FE0B40200400B31
:105ABE00C27285595A755C00129B4CE5537024E5F1
:105ACE0050B551028027A851E6F5560853006F7065
:015ADE0006C1
:105ADF0086570853006F8851128B01E553600D757F
:105AEF00552075A0E8A855E2F81281C230730280E4
:105AFF000CE559B55A028005128D93D273E55C708F
:105B0F0011307318128CB6C273E55C600F755E2886
:105B1F00C27375A0E8A95EE3F812821F12814C10C0
:105B2F005D14105C061075210297CA128E8F449077
:105B3F00129B6F0297CA129B17F853000703543832
:105B4F004844C0129B6F0297CA7583E8E5744440BE
:105B5F00F582E0547F129B6F0297CA7583EAE57650
:105B6F004400F582E022C26B12855D307B1B1285EB
:105B7F0020B3921B201C05301B0F8003201B0AA291
:105B8F001B921C74A092E0716F90E83FE004F0222A
:105B9F001289B9C26F857674129B17F5791286999F
:105BAF00E57444FCF590D27BD2EC128520B3921BA6
:105BBF00921C22C0E075A0F47819E230E2FCD0E02C
:105BCF00781BF23001031285522275A0F47819E286
:075BDF0030E0FC781BE2221C
:025BE600071C9A
:025BE80062B6A3
:00000001FF
